:0200000480007A
:100000006F00C004732F2034930F8000630AFF0336
:10001000930F90006306FF03930FB0006302FF038A
:10002000170F0000130F8F2663040F0067000F00E7
:10003000732F203463540F006F00400093E19153FD
:10004000171F000023203FFC6FF09FFF732540F136
:1000500063100500970200009382020173905230F2
:10006000735000189702000093820202739052307E
:10007000B70200809382F2FF7390023B9302F0017B
:100080007390023A9702000093828201739052307B
:100090007350203073503030735040309301000063
:1000A00097020000938242F67390523013051000BD
:1000B0001315F501634C05000F00F00F93011000BC
:1000C0009308D005130500007300000093020000A0
:1000D000638E020073905210B7B2000093829210A8
:1000E0007390223073232030E39A62F4735000300F
:1000F00037250000130505807320053097020000A6
:100100009382420173901234732540F173002030C2
:1001100073D0013473250034930E30009301200016
:10012000631CD513F3F50034930E300093013000B7
:100130006394D51373660234930E2000930140003C
:10014000631CD611F3560134930E600093015000E6
:100150006394D6113725AD0B1305A5DEF3150534D1
:10016000930E2000930160006398D50F372500009F
:100170001305A5DE73350534B72EAD0B938EAEDEB9
:1001800093017000631AD50D37C500001305F5EE15
:1001900073250534B70EAD0B93018000631ED50B9C
:1001A00073250034B7CEAD0B938EFEEE9301900015
:1001B0006314D50B7325103013750502630805020F
:1001C000B765000073A00530530000F073B0053030
:1001D00097250000938505E327A0050003A50500EA
:1001E000930E10009301A0006318D50773251030FB
:1001F000135545011375150063040504B72200006B
:100200009382028073B00230970200009382020151
:1002100073901234730020301305F00F731500C073
:10022000930EF00F9301B0006318D5031305F00F80
:1002300073250030930EF00F9301C000631ED501AB
:100240000F00F00F930110009308D0051305000074
:1002500073000000631030020F00F00F6380010094
:100260009391110093E111009308D00513850100CB
:10027000730000000F00F00F930110009308D005E9
:1002800013050000730000009302900063E6510024
:100290009302B00063F23202F32220341303800091
:1002A000E39C62FA0F00F00F930110009308D00551
:1002B0001305000073000000F32220341303200014
:1002C000E39C62F8F322103493824200739012345C
:1002D00073002030731000C0000000000000000018
:1002E000000000000000000000000000000000000E
:1002F00000000000000000000000000000000000FE
:1010000000000000000000000000000000000000E0
:1010100000000000000000000000000000000000D0
:1010200000000000000000000000000000000000C0
:1010300000000000000000000000000000000000B0
:081040000000000000000000A8
:1020000001000000000000000000000000000000CF
:040000058000000077
:00000001FF
